:020000040000FA
:020000000728CF
:04000A00003400348A
:02000E000730B9
:100010009F008316D73081008B0180308600FF302F
:10002000850083128601142805181428851A2728AC
:10003000051A362852203630860052203A30860083
:1000400052203930860052207530860014288518D9
:10005000382845203630860045203A308600452035
:1000600039308600452075308600142885182928E7
:1000700045207530860045203930860045203A30CD
:1000800086004520363086001428193005197D3049
:1000900085190A30A1008930A000A00B4D28A10BC2
:1000A0004B280800FA30A1008930A000A00B562888
:0E00B000A10B54281430A200A20B5C280800FB
:02400E00413F30
:00000001FF
